:020000040800F2
:10500000101A0020D55000084D8C000815840008A7
:105010000000000000000000000000000000000090
:10502000000000000000000000000000E1980008FF
:105030000000000000000000BD910008FD9900087C
:10504000E7500008E7500008E7500008E750000864
:10505000E7500008755B0008E7500008E7500008BB
:1050600000000000E7500008995A0008E7500008C7
:10507000E75000086D88000800000000E7500008B5
:1050800000000000E75000080000000000000000E1
:10509000E750000800000000E7500008E750000853
:1050A000E7500008E7500008E7500008D9A30008BF
:1050B000E7500008E7500008000000000000000072
:1050C0000348854600F060FC004800471DB2000818
:1050D000101A00200448804704480047FEE7FEE716
:1050E000FEE7FEE7FEE7FEE7999A0008C1500008D8
:1050F00030B50B46014600202022012409E00D4670
:10510000D5409D4205D31D469540491B25469540F7
:1051100040191546521E002DF1DC30BDF0B51FB40C
:105120000646002082B005464024019100901BE015
:10513000019922460F46304600F04EFB049A059B2B
:10514000801A994110D310461946224600F034FBCC
:10515000361A8F410197224601200021009F00F05E
:105160002BFB38184D4100902046641E0028DFDCE0
:10517000019B00982946324607B0F0BD03460B4319
:105180009B0703D009E008C9121F08C0042AFAD2FD
:1051900003E00B780370401C491C521EF9D2704783
:1051A000D2B201E00270401C491EFBD270470022BF
:1051B000F6E710B513460A4604461946FFF7F0FF16
:1051C000204610BD30B504460020034600E05B1CBD
:1051D000934203D2E05CCD5C401BF8D030BDF8B503
:1051E00002464A40D40F42004B0052085B089A42E4
:1051F00002D20246084611464A0023D0C30D4A0097
:10520000DDB2120EAD1A202D35DA49020126490A07
:10521000F6058A19002C00D0524220214F1B11465E
:10522000B9402A411018C20D9A4221D0002C17D043
:10523000012D08DCDA05801AD20F8019D207DBB203
:1052400000F0F6FAF8BDDA05801A012340001B06CB
:10525000C01880185A428018CA0F1043490007E04E
:105260004908C2071143DA05801A801940088018DE
:1052700000F0D6FAF8BD61000122511A001BF7E7D1
:105280000122D2075140AAE70122D2075040A6E7E7
:1052900070B502464A40D50F40004A00ED0740086D
:1052A0005208002814D0002A12D0C40DD30D410298
:1052B0000120C0055202490A520AE41A09181218BC
:1052C0007D34914201D3641C00E04900002C01DAD6
:1052D000002070BD0023914201D3891A0343400886
:1052E00049000028F7D100290AD0914202D10121BA
:1052F000C90705E0914201D2012101E00121C94322
:10530000E005C018401900F08BFA70BDF0B50746F3
:105310000846584087B0C00F049048000E46590018
:1053200040084908BC1A884105D2384631461E4615
:1053300017460B4602465800400810434CD0300D2B
:10534000039040055900400D490D0590401A029008
:10535000402872DA18030121000B09050843019067
:1053600004980092002805D00199524200208841FB
:1053700000920190029840210A1A0199009800F0C9
:105380001BFA05460C466B4607CB00F036FAC019EF
:105390007141039A0E0D0023D71756401A467A40E2
:1053A000164344D0049A002A2DD0029A012A039A67
:1053B00015DC1205C01A914101263605001C714109
:1053C000D20F059ED2070093019202962A462346E9
:1053D00000F074FA07B0F0BD38463146FAE716051A
:1053E000224A0F46B218C01AB74101210905001C14
:1053F0004F4100187F41114618187941E20F1043C0
:105400006D19644113E0E2076D0815436408C20793
:105410001443039A01261205C01A91413605001C57
:105420007141CE07400830434908C01851412A460F
:10543000234600F036FACDE7FFE70498012240004A
:10544000C117121A00238B4104983146C417381A29
:10545000A141EEE730B40124E407634030BC55E7D6
:1054600030B40124E407614030BC4FE70000E0FFA6
:10547000F0B51FB488B00B990998002448400999E9
:10548000C00F490049080991C0070B9900904900D5
:1054900049080B9109990898A64608431CD00B9916
:1054A0000A98084318D0099801244000420D48008A
:1054B000410D099824050003000B204309900B9827
:1054C0000003000B20430B9050181C494018002289
:1054D00001901446104605E0002001460DB0F0BDD5
:1054E000032801DA034600E003239C46C11A0AAEF2
:1054F0000AE05F0008ADED5B4F00F75B7D430027DE
:10550000AA187C41491C5B1E6145F2DD410004ABD9
:105510005A522104120C0A43240C401C0828DFDBD9
:10552000019802900099704601910090059B049AA1
:105530000799069800F0C2F9D0E700000DFCFFFFC4
:10554000F0B50C465C4085B0E40FE40703944C00D2
:1055500000266408590094464908024602962243F0
:1055600021D062460A431ED06200570D4A000E0346
:105570002303550D012402462C492405781B1B0BDF
:10558000360B401823432643614600901C46501AB0
:10559000B44103D30098401C009002E09218009898
:1055A0005B41002803DA0020014605B0F0BD002071
:1055B000012109050746864611E064461D46141B75
:1055C000B54106D36546521BB341744607430C43AD
:1055D000A646CD0740084908284392185B41054676
:1055E0000D43EAD11046184313D060461946504087
:1055F0007140084306D06046101AB34106D201221A
:10560000002306E000220123DB0702E00122D2434F
:105610005310009874460105381C6141029C039D9B
:105620000019694100F03DF9BFE70000FD030000EB
:10563000C217C10F504010B54018CA079623002169
:1056400000F0F6F810BD10B500229623114600F0C8
:10565000EFF810BD0EB5C217C10F5040CA07401871
:105660000021054B0293019200910A460B4600F07F
:1056700025F903B000BD0000330400000EB5054954
:105680000291002100910A460B46019100F016F9A3
:1056900003B000BD33040000410040020122400A73
:1056A000D205090E80187F2901DA0020704796295B
:1056B00003DC9622511AC8407047963988407047DB
:1056C00070B5CD0F4A0009030123090B1B051943CF
:1056D0000B4BED070024520D9A4201DA002070BDF9
:1056E000074B34339A4203DC9A1A00F075F802E053
:1056F0000449511888402C43F1D0404270BD00004D
:10570000FF030000CDFBFFFF4A0009030123090B43
:105710001B051943094B10B5520D9A4201DA0020BE
:1057200010BD064B34339A4203DC9A1A00F054F849
:1057300010BD03495118884010BD0000FF03000050
:10574000CDFBFFFFC20FD207400040080BD0C10DB8
:105750000723DB01C91840020905400A1143C208AA
:10576000400711437047002001467047CB0FDB070D
:10577000490010B5490802460A4307D00A0D07241C
:105780000903E401090B121B002A01DC002010BDF3
:10579000C900440F0C43C100E018D205801800F086
:1057A0003FF810BD0122D207002800DB101A0029A3
:1057B00000DB511A8142704710B5202A04DB0146F4
:1057C000203A9140002010BD914020239C1A0346AE
:1057D000E3401943904010BD10B5202A04DB084671
:1057E000203AD040002110BD0B46D340D0402024A9
:1057F000A21A91400843194610BD10B5202A06DBB5
:10580000CB170846203A1041C1170B4306E00B4660
:105810001341D0402024A21A91400843194610BDDC
:10582000002904DA401C490001D1400840007047BB
:1058300070B40024050C05D11024000402D1002905
:1058400021D01124050E01D100020834050F01D129
:105850000001241D850F01D18000A41C002801DB5C
:105860004000641C002908D020252E1B0D46F54061
:10587000A14000D001212943084301061B1B000A57
:10588000DB1D02D5002070BC7047DB05181880189E
:105890000029F8DA401C4900F5D170BC40084000EE
:1058A000704710B5002B08DA0024401C61419218A3
:1058B0005B411A4301D14008400010BDF0B51FB450
:1058C00082B005460C0003D0084604F045FE02E015
:1058D00004F042FE20300246009021462846FFF7A1
:1058E0006BFF049B059A04460F4618431143084377
:1058F00014D0184610431BD0009840210A1A1846AD
:105900000599FFF769FF05460E46009A0599049828
:10591000FFF752FF084305D0012004E02046394636
:1059200007B0F0BD0020C11705430E432C43374399
:1059300000990E986305401A7905E40A00220C4389
:10594000FD0A0A3002D500200146E9E701051019D9
:1059500069410C9C0D9D00196941FFF7A2FFDFE72B
:1059600010B5002904DB0124E40740428C412146A4
:10597000002B04DB1C460123DB075242A341994262
:1059800000D1904210BD0000064C0125064E05E0F6
:10599000E36807CC2B430C3C98471034B442F7D350
:1059A000FFF792FB8CB50008ACB5000838B504468B
:1059B000074908480068FFF79BFB6043009002E03E
:1059C0000098401E009000980028F9D138BD0000D2
:1059D00040420F000C01002070B5044600252068ED
:1059E00080688007800F012807D120680068C00701
:1059F000C00F002801D0012000E00020002839D18C
:105A0000206880681C490840002801D1012000E07E
:105A10000020002809D1606D102108436065A06D49
:105A200001210843A065012070BD20688068012124
:105A30000843216888600120FFF7B8FF01F05EF994
:105A400005460EE001F05AF9401B0A2809D9606D9D
:105A5000102108436065A06D01210843A065012065
:105A6000E2E720680068C007C00F012148404840B5
:105A70000028E7D00020D7E71700008010B50023EA
:105A80001A4603E0845CE3189BB2521C8A42F9D3A5
:105A9000D84380B210BD000010B5034800F028FEC6
:105AA000024800F025FE10BDB0150020681500204A
:105AB00030B51C25446C2C400125A540046C656064
:105AC000046863608468102C04D10468A2600468D0
:105AD000E16003E00468A1600468E26030BD00009A
:105AE0001449012048720A4602205E325072032097
:105AF0003C3A507204200E3A50720F480D4B007819
:105B0000087022310870203108770C495A1C087837
:105B10005871497899712333187159712033187766
:105B20005977107551751A461E32107551751076D9
:105B30005176704740110020C7000020E40000208B
:105B400010B503F0A5FE202003F04EFF012005F064
:105B5000CBF8002003F048FF044804F069FF044834
:105B600005F00CFA002005F041FA10BDB00000204D
:105B70008380000070B505200121000701F0AAF81C
:105B80000025154C002800D06560144E02213046D7
:105B900001F0A0F8002817D1012020707F20C00557
:105BA000A0600F48808F002805D0012100228902C3
:105BB000304601F09CF80B48656000880A21484394
:105BC0000949088004F01AFC012000F07DFF022042
:105BD00000F07AFF70BD0000FC00002000040050BF
:105BE000400D0020D4000020E0000020704700009D
:105BF00000210A4A51610A494968012252021143AF
:105C0000074A51601146496808221143044A51600D
:105C10000021C209D201116070470000F815002070
:105C2000002002407FB500250C460646039500F093
:105C300003FFE009029003A901960095684600F071
:105C40007DFE002804D000F0BFFE002004B070BD2F
:105C500000F0BAFE0120F9E710B5002302E0C45CB1
:105C6000CC545B1C9342FAD310BD0000002039498C
:105C70008969FF2201321140914208D136494969B0
:105C800002221143344A5161FF2101310843314955
:105C90008969012252021140914208D12E49496975
:105CA000012211432C4A516101214902084329492B
:105CB0008969012292021140914208D1264949691D
:105CC00008221143244A51610121890208432149D4
:105CD00089690122D2021140914208D11E494969C5
:105CE000042211431C4A51610121C9020843194988
:105CF0008969012252031140914208D1164949692C
:105D000010221143144A51610121490308431149EA
:105D10008969012252041140914207D10E49496913
:105D2000202211430C4A5161202108430949896905
:105D3000012212041140914208D1074949694022C9
:105D40001143054A51610121090408430149886151
:105D50007047000000200240F815002070B504468E
:105D600000F0CCFF05460BE0601C002808D0002C9A
:105D700004D000F0C3FF401BA04201D9032070BD36
:105D80001F488069C007C00F0028EDD11C488069FA
:105D900002210840022801D1194988611848806908
:105DA000FF2101310840884223D01548806949000D
:105DB000084088421DD01248806949000840884246
:105DC00017D00F48806949000840884211D00C481C
:105DD00080698900084088420BD009488069090120
:105DE0000840884205D0064880694910084088422A
:105DF00003D1FFF73BFF0120C1E70020BFE7000010
:105E000000200240F8B51746002605460C4600F073
:105E100013FE09E029460220226800F0E5FD002873
:105E200004D1241D2D1D361DBE42F3D300F0CCFD40
:105E3000BE4201D20020F8BD0120F8BD10B50849CE
:105E400002460020054B497905E044001C5B944262
:105E500003D0401CC0B28842F7D310BD68120020A6
:105E60004800002010B500F03EFF10BD10B50948F5
:105E700001F040F980B2FFF701FC074A074BFFF73A
:105E8000F7FA0022064BFFF75BFBFFF73DFC80B201
:105E900010BD000060140020F853E3A59B843E4031
:105EA00000408F4070B5384C3648217F0175617FC6
:105EB000417536490A78027649784176314905209C
:105EC000133148720A2005F049F87D20C00005F022
:105ED0005FF82C49002213310C2005F029F900212C
:105EE0000C2005F037F9022005F088F8284D002134
:105EF0000F2004F0B3FF2842E062F8D0E06A411CB2
:105F000030D0400430D58122D20100210F2005F08D
:105F1000E4F80021102004F0A1FF41061948490EC1
:105F20000022633004F0D0FF164D6335687A0528EF
:105F300017D102221549681DFFF744F9002810D136
:105F40001148AE7C66710422691C4030FFF716F9D7
:105F500029461331084672005130FFF70FF903202C
:105F6000207070BD02F0B0FE0A480188608B0546C3
:105F7000FFF7BEF808480088414308486D1E0180BD
:105F8000658370BDA111002048000020E4000020BE
:105F900000D02724D0000020CE000020CC0000201C
:105FA00010B5084800F03AFB0A21064800F0C0FA94
:105FB000044800F06FF9800503D5024800F06DF940
:105FC00080B210BD04140020F8B52F4D002201212D
:105FD000284600F08CFEFFF7E3FFFFF734FB2B4E63
:105FE0003146FFF755F92A4C0122A0601146284698
:105FF00000F07DFE2749A068002588423EDB20781E
:10600000254F002815D02570FFF7CAFFFFF71BFBAF
:106010003146FFF73DF9A060FFF794FB00223B46B5
:10602000FFF718FA00221D4BFFF722FAFFF79EFB3D
:106030006060A068FFF786FB00223B46FFF70AFA84
:10604000174A184BFFF714FA06460F466068FFF729
:1060500079FB134A144B5242FFF70AFA32463B4689
:10606000FFF754F9FFF782FB10496060884201DDB9
:10607000616004E0FF21C905C84200D36560606823
:10608000FFF70AFBC0B2F8BD0004005000401B44FB
:10609000240000200000604000000C4000E064404C
:1060A0003333333333B33040CCCCEC3F0000C84201
:1060B000F8B5044600250026002700BF5020005DEB
:1060C000012801D10220F8BD01215020015500BF57
:1060D000206880688007800F012806D1206800684A
:1060E0000840002801D0012000E00020002841D114
:1060F000606DFF21013188430221084360652068FB
:10610000C0688707BF0F2068C068800880002168CA
:10611000C860206880680121C90708432168886039
:1061200000F0ECFD064611E000F0E8FD801B0A28B7
:106130000CD9606D0221884310210843606500BFBF
:1061400000215020015500BF0120BCE72068806875
:10615000C00FC0070121C9078842E5D02068C06888
:1061600038432168C860606D0221884301210843DB
:10617000606504E0606D202108436065012500BF73
:1061800000215020015500BF28469CE770B5044609
:106190000D4600BF5020005D012801D1022070BDD6
:1061A00001215020015500BF20688068042108406B
:1061B000800800280AD0606D20210843606500BF78
:1061C00000215020015500BF0120E8E72D496868F3
:1061D000884229D02068806A29684903490B08430E
:1061E0002168886228684003400B27490840012144
:1061F0008904884208D12548806849010843234919
:1062000088600A20FFF7D2FB28684003400B204932
:1062100008400121490488422CD11C48806849016A
:1062200008431A49886025E02068806A2968490384
:10623000490B88432168886228684003400B124953
:10624000084001218904884205D11048806849012D
:1062500088430E49886028684003400B0C49084079
:1062600001214904884205D10848806849018843D2
:106270000649886000BF00215020015500BF002062
:106280008DE70000011000000000044800270140D5
:10629000000002440146486D704701460868006CE2
:1062A0007047000010B50446002C01D1012010BD3C
:1062B000606D002806D1A0650021502001552046C0
:1062C00000F00EF9606D10210840102806D02068FB
:1062D000806804210840800800280AD0606D1021E1
:1062E0000843606500BF00215020015500BF012018
:1062F000DDE7606DFF2101318843022108436065BD
:10630000206880688007800F012807D12068006816
:10631000C007C00F002801D0012000E000200028A5
:106320003AD100BF032189076068884207D04942FB
:106330006068884203D04900606888420CD12068B8
:106340000069800080082168086120680069616830
:1063500008432168086112E0206800698000800815
:10636000216808615C4880680F21890488435A4984
:10637000886008468068616808435749886000BFA4
:106380002068C068182188432168C8602068C068F8
:10639000A16808432168C8604F4880680121490608
:1063A00088434D49886008468068A18E49060843A5
:1063B0004949886020688068012109070840002851
:1063C00004D1206880680843216888602068C0681C
:1063D000424908402168C8602169E068022901D16A
:1063E000042100E0002108432021095D49030843FE
:1063F0002C21095D49000843216B0843A1698903E9
:106400000843E169C90308432168C9680843216852
:10641000C860FF21C231606A884207D0A16A606A01
:1064200008432168C96808432168C8602120005DCD
:10643000012813D12020005D002807D12068C06802
:106440000121090408432168C86007E0606D20212C
:1064500008436065A06D01210843A065E06B012839
:1064600017D120680069FF218900884321680861ED
:10647000216C606C0843A16C0843216809690843DA
:1064800021680861206800690121084321680861CA
:106490000BE020680069C007C00F002805D0206805
:1064A0000069400840002168086120684069C00810
:1064B000C0002168486120684069A16B08432168D9
:1064C00048610020A065606D0221884301210843D6
:1064D00060650020EBE60000002701401902FEFF86
:1064E00010B586B0044614216846FEF760FE0E49DA
:1064F0002068884216D10D48416B42151143416313
:10650000C16A01221143C162C06A69461040059008
:106510000220009003200190002002900520000737
:1065200000F0E2FA06B010BD002401400010024065
:10653000F8B504460D46002600276069082801D1F9
:10654000082711E02068C068C007C00F00280AD0E3
:10655000606D20210843606500BF00215020015577
:1065600000BF0120F8BD0C2700F0C8FB064614E070
:10657000681C002811D0002D04D000F0BFFB801B48
:10658000A8420AD9606D04210843606500BF00215C
:106590005020015500BF0320E4E720680068384020
:1065A0000028E5D0606D012149020843606520683C
:1065B000C068032189020840002826D12020005D00
:1065C000002822D1206800680821084008281CD132
:1065D0002068806804210840800800280DD12068C8
:1065E00040680C21884321684860606DFF210131BB
:1065F000884301210843606507E0606D202108435E
:106600006065A06D01210843A065A069002802D142
:106610000C20216808600020A4E7000070B5044643
:1066200000252068806804210840800800282BD1BC
:1066300000BF5020005D012801D1022070BD012162
:106640005020015500BFE069012803D02046FFF724
:10665000C3F90546002D18D1606D0D490840FF2192
:106660000131084360650020A06500BF0021502073
:10667000015500BF1C202168086020688068042143
:1066800008432168886000E002252846D6E700001C
:10669000FEF1FFFF70B5044600252520005D0228AD
:1066A00003D00420E063012520E0206800680E216B
:1066B000884321680860206800684008400021681D
:1066C00008601C21606C084001218140206C416001
:1066D00001212520015500BF00212420015500BFC4
:1066E000A06B002802D02046A16B8847284670BDC9
:1066F00070B50446206C0568206806681C20616C33
:10670000014004208840284000281DD0042030404B
:10671000002819D02068006820210840002805D1F1
:106720002068006804218843216808601C21606C8F
:10673000084004218140206C4160206B00285AD021
:106740002046216B884756E01C20616C01400220E6
:1067500088402840002825D002203040002821D041
:106760002068006820210840002808D120680068BF
:106770000A218843216808600121252001551C2138
:10678000606C084002218140206C416000BF002104
:106790002420015500BFE06A00282CD02046E16A81
:1067A000884728E01C20616C014008208840284070
:1067B000002820D00820304000281CD02068006825
:1067C0000E218843216808601C21606C084001216B
:1067D0008140206C41600120E063012125200155AA
:1067E00000BF00212420015500BF606B002802D0AB
:1067F0002046616B884770BD70B50446002C01D1FE
:10680000012070BD244A2168881A1421FEF770FC0B
:10681000800060642048083820640221252001554A
:10682000206805681D480540E168A06808432169A3
:10683000084361690843A1690843E1690843216A83
:10684000084305432068056001218903A068884248
:1068500017D011487830806A1C22616C11400F22D9
:106860008A4090430C49783188621C22616C114047
:106870006068884008497831896A08430649783158
:1068800088620020E0630121252001550021242099
:1068900001550020B5E70000080002400F80FFFF0F
:1068A000F8B504460D4616461F460020009000BF6E
:1068B0002420005D012801D10220F8BD01212420FF
:1068C000015500BF2520005D01282DD10221252082
:1068D00001550020E06320680068400840002168FE
:1068E00008603B46324629462046FFF7E1F8206B18
:1068F000002806D0206800680E210843216808603F
:106900000BE0206800680421884321680860206843
:1069100000680A2108432168086020680068012196
:1069200008432168086006E000BF002124200155CB
:1069300000BF022000900098BFE70000F8B50446B1
:106940000E460127002500BF1C48007C012801D10C
:106950000220F8BD01201949087400BF1848FFF74C
:10696000FDF90746002F22D1401E3060656817E010
:106970002846FFF73DF91248FFF7F0F9074611489E
:106980004068082188430F49486008464068491517
:1069900088430C494860002F01D0356006E08035FF
:1069A000A068C00161684018A842E1D800BF00BFDC
:1069B00000200249087400BF3846CAE7F8150020D5
:1069C00050C30000002002400648406802210843EE
:1069D000044948600846406801210843014948606D
:1069E0000020704700200240F8B507460C461546C7
:1069F000012600BF0E48007C012801D10220F8BD0D
:106A000001200B49087400BF0A48FFF7A7F90646A2
:106A1000002E06D10649486125600648FFF79EF919
:106A2000064600BF00200249087400BF3046E6E772
:106A3000F815002050C300001D484068C007C00F73
:106A4000002816D000BFEFF31080014600BF72B6D9
:106A50001848174AD0601848D06000BF81F31088EA
:106A600000BF10464068C007C00F002801D00120B9
:106A700070470F48406802221040022815D100BF1D
:106A8000EFF31080014672B60C48094A10610C48B9
:106A90001061084680F3108800BF1046406802224B
:106AA0001040022801D10120E2E70020E0E70000C9
:106AB00000200240EFCDAB8905040302BFAE9D8CE0
:106AC000161514137047000010B5044605484069B8
:106AD0002040002804D0034844612046FFF7F2FF1D
:106AE00010BD00000004014070B5034600220024E0
:106AF0000020DAE0012696400D6835402C46002C37
:106B000077D04D68022D02D04D68122D15D1D508D1
:106B1000AE001D462035A8595507EE0E0F25B5408D
:106B20000646AE4330465607F60E0D69B54028437B
:106B3000D508AD001E46203670514D68012D08D095
:106B40004D68022D05D04D68112D02D04D68122DD3
:106B500018D1986856000325B5400646AE43304626
:106B60005600CD68B5402843986058680125954087
:106B70000646AE43304610264D6835402D099540F7
:106B800028435860186856000325B5400646AE43B2
:106B900030460D79AD07AD0F5600B540284318605B
:106BA000D86856000325B5400646AE433046560029
:106BB0008D68B5402843D860012636074D683540BA
:106BC000B54271D13C4D6D6B012635433A4E75632C
:106BD0003A4D9608B600A85995072E0F0F25B540D7
:106BE0000646AE43304605252D07AB4202D10025AF
:106BF00015E059E0324DAB4201D101250FE0314D96
:106C0000AB4201D102250AE02F4DAB4201D1032551
:106C100005E02E4DAB4201D1052500E00625960783
:106C2000360FB5402843254D9608B600A851284D8B
:106C300028680546A5432846012636044D68354098
:106C4000B54202D1054625432846214D2860686893
:106C50000546A5432846012676044D683540B542D1
:106C600002D1054625432846194D6860A8680546A7
:106C7000A5432846012636054D683540B54202D168
:106C8000054625432846124DA860E8680546A543F9
:106C90002846012676054D683540B54202D10546A5
:106CA000254328460A4DE860521C0D68D540002D4A
:106CB00000D01FE770BD0000001002400800014036
:106CC0000004005000080050000C0050001C005050
:106CD00000040140024613690B40002B01D0012043
:106CE00000E00020704742694A4042617047002A34
:106CF00001D0816100E081627047000001480068B6
:106D0000704700000801002002480068401C01494B
:106D1000086070470801002010B50024084800688A
:106D20004021084306490860002000F00BF80028C5
:106D300001D0012401E000F013FA204610BD00004C
:106D40000020024070B5044600257D21C900094895
:106D50000068FEF7CDF9064601F0B6F8002801D02C
:106D6000012504E000222146501E00F01DFA2846AD
:106D700070BD00000C01002070477047F8B5394C19
:106D80000126A078401CA0702671E08A401CE08299
:106D90003548008802F0E2FD344DE888FEF753FCE8
:106DA0003349FEF775FA334F3968FEF718FA386041
:106DB0003148F105006800270090884210DB208AE6
:106DC000FEF741FC01467F20C005FEF761FA0099FD
:106DD000FEF75AFA2849086028480221017001E0AC
:106DE0002648077002212648FFF774FF002809D0C3
:106DF00027632048234A016823480091914212DD0D
:106E0000067011E0E888FEF71EFC1949FEF740FA0B
:106E1000216BFEF7E4F91B4920638842E9DB1C493A
:106E20001A48C860E5E70770688F401EFEF700FC4F
:106E30000099FEF7B7FC05D86079002802D0154804
:106E4000067001E013480770688FFEF7FCFB0949E4
:106E50000968FEF7A7FC04D26079002801D004F08D
:106E600069FAF8BDC400002062000020400D002037
:106E700000007A4400010020040100205900002095
:106E8000000400500000F0424E0000200400FA050B
:106E900000ED00E05B000020704710B50446002CB8
:106EA00001D1012010BD02212E200155204601F004
:106EB000E5FC204600F0F4F800212E20015500BF2B
:106EC0002D20015500BF0020ECE77047704710B53A
:106ED000044620680068C007C00F012148404840B0
:106EE00000280CD0206880680840484048400028AE
:106EF00005D00120216848602046FFF73FFF206849
:106F0000006802210840400800280BD020688068F3
:106F100008404008002805D002202168486020462B
:106F2000FFF72AFF20680068042108408008002835
:106F30000BD02068806808408008002805D0042015
:106F400021684860204600F009F92068006808219F
:106F50000840C00800280BD0206880680840C0089E
:106F6000002805D00820216848602046FFF794FFDC
:106F70002068006810210840000900280BD0206814
:106F8000806808400009002805D01020216848606A
:106F90002046FFF7F2FE20680068202108404009E3
:106FA00000280BD02068806808404009002805D0E0
:106FB0002020216848602046FFF788FF206800688D
:106FC00040210840800900280BD0206880680840D4
:106FD0008009002805D04020216848602046FFF73E
:106FE00074FF10BD70B50446002C01D1012070BDA6
:106FF0006068012800D100BF26496069884200D03E
:1070000000BF2E20005D002805D100212D20015554
:10701000204600F057F802212E2001552068C5684F
:107020006068012803D08905A06A884203D11E2127
:1070300028468843054617496069884201D01648AA
:10704000054016480540A16860680843216A084366
:10705000616A0843A16A084305436068012804D0B7
:107060000121C905A06A884203D1E168206908436B
:10707000054308496069884205D06169A0690843F1
:10708000E169084305432068C56001212E200155B0
:107090000020ACE7FFFF00003F1FFFFFF8F119FFE2
:1070A00010B500680549884207D10548816B490041
:1070B000490881630D2000F05FF810BD007C00409E
:1070C0000010024010B50068084988420CD10848F9
:1070D000816BC20411438163002201210D2000F065
:1070E00063F80D2000F054F810BD0000007C004053
:1070F0000010024001460868C069704710B5034699
:1071000002242E20C4541448006824072043124C43
:1071100020601868C0680124E40420431C68E06013
:1071200018688068012420431C68A0601868006902
:10713000012420431C68206118688161186842613D
:1071400018680069042420431C68206101242E2053
:10715000C454002010BD000000040140704700002E
:107160000448416B012211434163816B02041143C6
:10717000816370470010024000BFC206D20E012199
:107180009140024A116000BF7047000080E100E0BA
:1071900000BFC206D20E01219140024A116000BF19
:1071A0007047000000E100E070B504460D46164649
:1071B0002946204601F04CFD70BD00000249496897
:1071C0008143014A516070470070004003480068E5
:1071D000FF210131084301490860704700700040F9
:1071E000024949680143014A5160704700700040FC
:1071F00007480068022108430549086005480069FE
:10720000042108430349086100BF00BF30BF704735
:107210000070004000ED00E010B5024600200E4B6B
:107220001868800880000346134318460A4B18600C
:107230000A4B1B6904242343084C2361012901D113
:1072400030BF02E040BF20BF20BF044B1B690424B5
:10725000A343024C236110BD0070004000ED00E02C
:10726000F8B5044620212068084020287CD12068F9
:107270000840202800D100BF00278148806B0121F1
:1072800009070840002805D17D48806B08437C49E8
:10729000886301277B480068FF21013108400028EE
:1072A00016D178480068084376490860FFF726FD44
:1072B000064606E0FFF722FD801B642801D9032063
:1072C000F8BD70480068FF21013108400028F1D066
:1072D0006B480568032109050D4060680840A84215
:1072E0000DD0091160680840884208D164480068E0
:1072F000012149040840884201D10120E0E76048AB
:10730000403000690321090408400546002D3DD0A6
:1073100060680840A84239D0202120680840202811
:1073200034D1574840300069032109048843054699
:107330005348403000690121C90408435049403195
:107340000861084600690121C90488434C4940315D
:10735000086108460561801528408915884215D1C5
:10736000FFF7CCFC064608E039E0FFF7C7FC801BBE
:107370004549884201D90320A2E7414840300069CD
:10738000012149020840400A0028EED000BF00BF9A
:10739000032109046068084088420AD1384800681F
:1073A00009018843032212056168114008433449EA
:1073B000086000BF3248403000690322120461684F
:1073C000114008432E494031086100BF012F05D10B
:1073D0002B48806B890588432949886300BF207842
:1073E000C007C00F002809D025484030C068800879
:1073F0008000A168084322494031C860022120680A
:107400000840022809D11E484030C0680C2188433A
:10741000E16808431A494031C860042120680840E7
:1074200004280AD116484030C068032189028843E5
:107430002169084312494031C8600821206808408A
:1074400008280AD10E484030C06803210903884348
:10745000616908430A494031C860802120680840BA
:1074600080280AD106484030C06803218904884337
:10747000A169084302494031C860002020E70000AC
:10748000001002400070004088130000F8B5044668
:107490000D46002C01D10120F8BD79480068C007D5
:1074A000C00FA8420ED2764800684008400028432A
:1074B0007349086008460068C007C00FA84201D0A1
:1074C0000120E9E7022120680840022807D16D4821
:1074D000C068F0218843A16808436A49C8602078E1
:1074E000C007C00F00284CD06068022809D1654849
:1074F0000068012149040840400C002824D10120E3
:10750000CAE76068032809D15E480068012149067E
:107510000840400E002817D10120BDE7606801280F
:1075200008D15848006804210840800800280BD181
:107530000120B1E753480068012149020840400A90
:10754000002801D10120A7E74E48C06880088000CC
:10755000616808434B49C860FFF7D0FB0646606886
:1075600002280FD107E0FFF7C9FB801B464988427C
:1075700001D9032090E74348C0680C21084008283F
:10758000F1D134E0606803280FD107E0FFF7B6FBC4
:10759000801B3D49884201D903207DE73948C068F6
:1075A0000C2108400C28F1D121E0606801280FD19E
:1075B00007E0FFF7A3FB801B3349884201D9032072
:1075C0006AE73048C0680C2108400428F1D10EE079
:1075D00007E0FFF793FB801B2B49884201D903206A
:1075E0005AE72848C0680C2108400028F1D12448F7
:1075F0000068C007C00FA8420ED9214800684008A3
:10760000400028431E49086008460068C007C00FB4
:10761000A84201D001203FE7042120680840042847
:1076200008D11848C068072109028843E168084367
:107630001449C860082120680840082809D1114869
:10764000C0680721C90288432169C90008430D4960
:10765000C86000F049F80B49C968F02211400909D7
:107660000A4A515CC8400A4908600020FFF76AFBDB
:107670000746002F01D038460EE700200CE7000037
:107680000020024000100240881300006AB5000884
:107690000C01002001480068704700000C01002028
:1076A00000B5FFF7F7FF0549C9680722120211402C
:1076B000090A034A515CC84000BD000000100240A6
:1076C0007AB5000800B5FFF7E5FF0549C96807224C
:1076D000D2021140C90A034A515CC84000BD0000F3
:1076E000001002407AB50008FEB52E48C7680C208D
:1076F0003840002845D0042804D008280CD00C2895
:107700003ED10BE02748006810210840002801D036
:10771000254C00E0254C41E0254C3FE00F20800443
:107720003840800C23490E5C032080053840800DD2
:10773000401C01901B48C068012109040840002832
:1077400007D01B49714308460199FDF7D1FC054656
:1077500014E01448006810210840002807D012499E
:10776000714308460199FDF7C3FC054606E00F4941
:10777000714308460199FDF7BBFC05462C460DE018
:1077800000BF08484068072149030840400B0090AB
:107790000098401C01218140CC0300BF00BF20465F
:1077A000FEBD00000010024000093D000024F4006E
:1077B00000127A0082B50008FEB50446002C01D103
:1077C0000120FEBDF848C6680C210E40C7680121A3
:1077D00009040F402078C007C00F002872D0082E7F
:1077E00004D00C2E0FD1084687420CD1EE48006819
:1077F000012149040840400C002863D0606800283B
:1078000060D10120DDE700BF0121090460688842E2
:1078100005D1E54800680843E349086027E00521F1
:107820000904606888420ED1DF480068012189049C
:107830000843DD490860084600680121090408433F
:10784000D949086013E0D848006801210904884339
:10785000D5490860084600680121090408400090E5
:1078600000BFD148006889008843CF49086000BF45
:107870006068002813D0FFF741FA054606E0FFF7DD
:107880003DFA401B642801D903209AE7C6480068E6
:10789000012149040840400C0028F0D012E0FFF715
:1078A0002DFA054606E0FFF729FA401B642801D9A6
:1078B000032086E7BC480068012149040840400CC9
:1078C0000028F0D102212068084002287AD1E0681F
:1078D0000290042E03D00C2E34D1002F32D1B248A6
:1078E0000068042108408008002804D0029800287D
:1078F00001D1012065E7AC4840681F210902884397
:10790000216909020843A84948600846006809211E
:10791000884302990843A4490860FFF7E5FEA2499D
:10792000C968F02211400909A04A515CC840A04929
:1079300008600020FFF706FA01900198002841D066
:1079400001983EE70298002824D097480068092152
:1079500088430299084394490860FFF7CFF9054628
:1079600006E0FFF7CBF9401B022801D9032028E7E6
:107970008D4800680421084080080028F1D08A481A
:1079800040681F210902884321690902084386498A
:10799000486017E084480068400840008249086059
:1079A000FFF7ACF9054606E0FFF7A8F9401B0228EF
:1079B00001D9032005E77C480068042108408008BD
:1079C0000028F1D1102120680840102867D1002E2E
:1079D00036D17548006849010840400A002804D0A3
:1079E000A069002801D10120EBE66F48406807211B
:1079F00049038843216A08436B4948600846406848
:107A00000002000A217F0906084367494860206A8E
:107A1000400B401C01218140C8036349C968F02222
:107A200011400909614A515CC84061490860002061
:107A3000FFF788F90190019800284BD00198C0E623
:107A4000A06900282CD058480068FF210131084364
:107A500055490860FFF752F9054606E0FFF74EF971
:107A6000401B022801D90320ABE64F4800680121E2
:107A700049020840400A0028F0D04B4840680721DE
:107A800049038843216A08434749486008464068DB
:107A90000002000A217F090608434349486019E0B3
:107AA00041480068FF21013188433F490860FFF7E2
:107AB00025F9054606E0FFF721F9401B022801D908
:107AC00003207EE638480068012149020840400A48
:107AD0000028F0D1082120680840082839D16069C1
:107AE00000281BD0304840300069012108432E494E
:107AF00040310861FFF702F9054606E0FFF7FEF89E
:107B0000401B022801D903205BE62748403000696A
:107B10000221084040080028F0D01AE022484030F6
:107B2000006940084000204940310861FFF7E6F84D
:107B3000054606E0FFF7E2F8401B022801D90320C2
:107B40003FE61948403000690221084040080028FB
:107B5000F0D1042120680840042879D10020009049
:107B60001148806B89060840002806D10E48806BBA
:107B700008430D498863012000900E480068FF21EA
:107B80000131084000281ED10A480068084309490D
:107B90000860FFF7B3F805460EE0FFF7AFF8401BAB
:107BA000642809D903200CE6001002406AB50008D9
:107BB0000C0100200070004085480068FF21013161
:107BC00008400028E9D000BFFF210131A0688842A9
:107BD00005D18048006908437E49086130E0A0680B
:107BE00000280DD17B480069FF2101318843794984
:107BF00008610846006909158843764908611FE055
:107C000005210902A06888420DD17248006901214E
:107C1000890208436F4908610846006989150843CD
:107C20006C4908610CE06B480069FF210131884311
:107C30006849086108460069091588436549086173
:107C400000BFA068002815D0FFF758F8054608E0E7
:107C500031E0FFF753F8401B5F49884201D9032008
:107C6000AFE55C480069012149020840400A00284C
:107C7000EFD013E0FFF742F8054607E0FFF73EF8C4
:107C8000401B5549884201D903209AE551480069B3
:107C9000012149020840400A0028EFD1009801283C
:107CA00008D14C484038806B012109078843494975
:107CB0004039886300BF606A00284CD00C2E69D020
:107CC000606A022848D1434840380068012109060B
:107CD0008843404940390860FFF710F8054606E040
:107CE000FFF70CF8401B022801D9032069E5394849
:107CF00040380068012149060840400E0028EFD1B5
:107D0000E16AA06A0843216B084332494039C968D7
:107D1000FD221204914308432E494039C8600846A9
:107D200000680121090608432A4940390860FEF726
:107D3000E5FF054606E0FEF7E1FF401B022801D9FA
:107D400003203EE5234840380068012149060840E9
:107D5000400E0028EFD038E01E484038006801216E
:107D6000090688431B4940390860FEF7C7FF0546EE
:107D700006E0FEF7C3FF401B022801D9032020E5DF
:107D8000144840380068012149060840400E002888
:107D9000EFD11AE0606A012800D112E50D484038A1
:107DA000C768012000043840A16A88420BD10F2027
:107DB00080043840E16A884205D1032080053840BC
:107DC000216B884201D00120FBE40020F9E400008F
:107DD00000700040401002408813000010B50446B7
:107DE000002C01D1012010BD606A002800D100BF25
:107DF0000021A1625120005D002804D150200155CE
:107E0000204600F035F80221512001552068006815
:107E10004021884321680860A16860680843E168E0
:107E20000843216908436169084301225202A1699C
:107E300011400843E1690843216A0843A16A0843E5
:107E400021680860A069000C04210840616A0843A9
:107E5000216848602068C069910088432168C86132
:107E6000002060650121512001550020BBE7000082
:107E700010B586B0044614216846FDF798F91049FC
:107E80002068884219D10F48416B82141143416325
:107E9000C16A01221143C162C06A002110400590ED
:107EA000E0200090022001900320039002910491B1
:107EB000052069460007FEF717FE06B010BD00005A
:107EC000003001400010024070B504462546681E8F
:107ED0000949884201D901200CE0681E0749486120
:107EE0000321081F00F0B4FE002004498861072028
:107EF0000861002070BD0000FFFFFF0000E000E00F
:107F000070477047FEB504462068C569206806685A
:107F1000206887682807000F0190019800280ED17B
:107F20002020284000280AD020203040002806D0F9
:107F3000206E002802D02046216E8847FEBD0198A1
:107F400000287DD0F807C00F002804D1FF20213081
:107F500030400028F5D0E807C00F00280BD0FF20E4
:107F600001303040002806D0012021680862E06F0F
:107F700001210843E0670220284000280AD0F807C2
:107F8000C00F002806D0022021680862E06F04219B
:107F90000843E0670420284000280AD0F807C00FF3
:107FA000002806D0042021680862E06F02210843FF
:107FB000E0670820284000280ED02020304000280C
:107FC00003D1F807C00F002806D0082021680862F6
:107FD000E06F08210843E067E06F002846D02020CA
:107FE0002840002809D020203040002805D0206EED
:107FF000002802D02046216E8847E06F009020685C
:10800000806840210840402804D00821009808409A
:10801000002826D0204601F05EFF206880684021BD
:108020000840402819D1206880688843216888600A
:10803000E06E00280DD02548E16E8863E06E00E018
:1080400015E0FEF727FB002810D0E06E816B884713
:108050000CE02046FFF755FF08E02046FFF751FFF0
:1080600004E02046FFF74DFF0020E06766E70120AF
:108070000005284000280CD0012080053840002849
:1080800007D001200005216808622046FFF738FF6D
:1080900054E78020284000280AD080203040002863
:1080A00006D0606E002802D02046616E884745E702
:1080B00040202840002807D040203040002803D02E
:1080C000204601F01AFF39E700BF37E7159E000888
:1080D00010B50446002C01D1012010BDA069002874
:1080E00000D000E000BF606F002805D100217020A3
:1080F0000155204600F02CF82420606720680068B5
:108100004008400021680860204601F041FF012836
:1081100000D1E2E7606A002802D0204601F042FD6B
:10812000206840680921C9028843216848602068A6
:1081300080682A21884321688860206800680121BE
:10814000084321680860204601F0A4FDC5E700004F
:10815000F0B587B0064614216846FDF728F82C498B
:108160003068884251D12B48416B01229203114360
:108170004163C16A01221143C162C06A00251040F7
:1081800005900320400200900220032701A9A1C10D
:1081900004200490052069460007FEF7A5FC1F4C4B
:1081A0001D48A560E56081C48027E560A7602020A8
:1081B000256160610002A0611848083CFEF71CFBC5
:1081C000002801D0FDF712FDF466A662144C124897
:1081D0002146143820600320606010200831A1C1BE
:1081E0006561A561E56120462562FEF705FB002873
:1081F00001D0FDF7FBFCB466002201211B20A66222
:10820000FEF7D2FF1B20FEF7C3FF07B0F0BD000052
:108210000038014000100240300002406815002084
:10822000B015002070B504460D461646A06F2028F4
:1082300063D1002D01D0002E01D1012070BD01219C
:108240000903A068884208D12069002805D1E80701
:10825000C00F002801D00120F0E700BF7020005DB2
:10826000012801D10220E9E701217020015500BF5A
:108270006565582006530020E0672220A067E06E65
:10828000002820D01E48E16EC8621E48E16E0863D7
:108290001D48E16E48630020E16E8863236819463B
:1082A00024313346626DE06EFEF7FAFA00280AD0F8
:1082B0001020E06700BF00217020015500BF202082
:1082C00060670120BAE700BF00217020015500BFA0
:1082D00020680068FF210131084321680860206898
:1082E00080680121084321688860206880684021F7
:1082F0000843216888600020A0E702209EE7000074
:108300007F9E0008C99E00082D9E00087047704798
:10831000FFB583B004460D461746606F202875D11F
:10832000002D01D0002F02D1012007B0F0BD0121A6
:108330000903A068884208D12069002805D1E80710
:10834000C00F002801D00120EFE700BF7020005DC2
:10835000012801D10220E8E701217020015500BF6A
:108360000020E06721206067FEF7C8FC01905020E4
:1083700007535220075301210903A068884205D101
:108380002069002802D10026029502E02E46002036
:10839000029021E006980090002280212046019B57
:1083A00001F0E4FF002801D00320BEE7002E09D130
:1083B00002980088C005C00D216888620298801C60
:1083C000029003E0307821688862761C5220005BBE
:1083D000401E81B2522001535220005B0028D9D1A7
:1083E00006980090002240212046019B01F0BEFF2C
:1083F000002801D0032098E72020606700BF0021FB
:108400007020015500BF00208FE7FFE702208CE7B6
:108410007047000001490248C160FDE70400FA0509
:1084200000ED00E010B505242407002204212046B9
:10843000FEF75DFC002208212046FEF758FC0A20CA
:1084400002F0AFFA012204212046FEF750FC0A2078
:1084500002F0A7FA002204212046FEF748FC10BDD6
:1084600010B505242407002204212046FEF73FFC16
:10847000012208212046FEF73AFC0A2002F091FA78
:10848000012204212046FEF732FC0A2002F089FA7C
:10849000002204212046FEF72AFC10BDF8B5002476
:1084A0000526074625463607002204213046FEF7FA
:1084B0001EFC0A2002F075FA012204213046FEF764
:1084C00016FC6006040E08213046FEF703FC002867
:1084D00001D0641CE4B2052002F063FA6D1CEDB219
:1084E000082DE1D3002F03D0FFF79CFF2046F8BDF5
:1084F000FFF7B6FFFAE770B50526054636070022F6
:1085000004213046FEF7F3FB0024E80901D00122E4
:1085100000E0002208213046FEF7E9FB6806050E60
:108520000A2002F03EFA012204213046FEF7DFFB6A
:108530000A2002F036FA002204213046FEF7D7FB6B
:108540000A2002F02EFA641CE4B2082CDDD370BDC0
:1085500010B505242407012208212046FEF7C7FB99
:10856000012204212046FEF7C2FB002208212046FA
:10857000FEF7BDFB0A2002F014FA00220421204677
:10858000FEF7B5FB10BD10B5052424070022042119
:108590002046FEF7ACFB002208212046FEF7A7FB91
:1085A0000A2002F0FEF9012204212046FEF79FFB7B
:1085B000012208212046FEF79AFB0A2002F0F1F979
:1085C00010BD70B505252D0700240122082128467D
:1085D000FEF78DFB062002F0E4F901220421284673
:1085E000FEF785FB062002F0DCF907E0641CE4B22C
:1085F000FA2C03D9FFF7C7FF012070BD08212846D8
:10860000FEF768FB0028F1D1002204212846FEF77E
:108610006EFB002070BD0000F8B501F073FB01F0A7
:10862000ADFB47480068C069464E474F800700D5FC
:10863000FE60FDF71BFC4549454C898F002914D08D
:1086400044490A7801218902002A0AD0012A04D06B
:10865000022A04D0032A08D103E0212801D20022F3
:1086600000E001222046FEF742FB0121C902384802
:10867000FEF730FB384C0025002824D03748056031
:10868000E079002803D10120E07101F0B7FE2078E5
:10869000632806D9002208212D48FEF728FB012275
:1086A00005E0012208212A48FEF721FB00220121D2
:1086B0000520C9030007FEF71AFB244C4034A08CA8
:1086C000012803D01CE0E5710022EBE7244869464D
:1086D000088072B680212348FDF7A4FA002804D050
:1086E000022269461F48FDF78DFB62B61EA001F00D
:1086F00023FFA58402F0BAFE642002F04BF9FE606D
:10870000608C012808D111486584058002F0AEFE16
:10871000642002F03FF9FE60208C012806D12584F8
:1087200002F0A4FE642002F035F9FE600748124A08
:108730000188914202D1C088002800D1FE60F8BDB6
:10874000E81400200400FA0500ED00E0400D0020D0
:108750000004005059000020C40000200001002047
:10876000AAAA0000384A0008BDF8C8EBC9FDBCB68B
:10877000C4A3CABD0D0A0000AA55000008B53721E0
:10878000202000F06EF80321212000F06AF840213B
:10879000222000F066F80821232000F062F8AA21C8
:1087A000302000F05EF80A48008FC1B2322000F09D
:1087B00058F80221332000F054F85F21202000F007
:1087C00050F8684600F006F80A2002F0EAF808BD02
:1087D000400D002010B501460F2000F021F80028C0
:1087E00000D0012010BD10B50446FFF7B1FE3220C5
:1087F000FFF781FEFFF7E5FEE0B2FFF77CFEFFF733
:10880000E0FEFFF7A5FE3320FFF775FEFFF7D9FE68
:108810000020FFF743FE0446FFF7B5FE204610BDDB
:1088200010B50C46FFF7DFFF2070012010BD70B5BA
:108830000D460446FFF78CFE3220FFF75CFEFFF783
:10884000C0FEE0B2FFF757FEFFF7BBFE2846FFF77A
:1088500052FEFFF7B6FEFFF796FE0A2002F0A1F8DF
:1088600070BD10B5FFF7E3FF012010BD10B5024841
:10887000FEF72DFB10BD000060140020F0B585B0A0
:1088800004460020039072B64F4920684018002823
:1088900006D14E48C068032189040840039000E0D7
:1088A00000BF00BF2068806802902068C068019007
:1088B0002068456920688669434920684018002877
:1088C0000DD142484038806A490508433F49403944
:1088D00088620846806A40004008886200E000BF65
:1088E00000BF002D01D1002E5FD03749206840180D
:1088F000002807D13548C0680321890488433349DB
:10890000C86000E000BF00BF002D1DD020680069D6
:10891000012108432168086120684561FEF7EEF9EE
:10892000074600BFFEF7EAF9C01B00902068006808
:1089300008210840082804D07D21C90000988842F9
:10894000F0D9082021684860002E1DD020680069F9
:10895000012108432168086120688661FEF7CEF98D
:10896000074600BFFEF7CAF9C01B009020680068E8
:1089700010210840102804D07D21C90000988842A9
:10898000F0D91020216848600F492068401800285D
:1089900009D10E48C068032189048843039908431C
:1089A0000A49C86000E000BF00BF206800694008B5
:1089B0004000216808610298216888600198216858
:1089C000C86062B605B0F0BD0084FFBF4010024031
:1089D0001CB5002116480091144A01910260C16340
:1089E0001205426081600722826301220261024611
:1089F000C16020321170FF235170C2334362816223
:108A0000117301638161042241634261C161FDF719
:108A100049FC084800908013019069460448FDF71E
:108A2000B5FB00210248FDF743FB1CBD00240140BB
:108A3000041400200200000408B50848016B01225C
:108A400011430163006B01211040009000220A20B5
:108A5000FEF7AAFB0A20FEF79BFB08BD00100240B0
:108A6000F0B587B014216846FCF7A1FB4C48C26AF8
:108A700004210A43C262C26A0A400592C16A802781
:108A80003943C162C16A39400591C16A0125294350
:108A9000C162C16A29400591C16A02263143C1629F
:108AA000C06A2A463040059005201C210007FEF7C9
:108AB0001EF901223B493C48FEF719F900223B49C7
:108AC0003948FEF714F99121052000220902000718
:108AD000FEF70DF9364801900024052069460095FF
:108AE00002940007FEF700F8032001900520694674
:108AF000009602940007FDF7F7FF0C20009011206C
:108B00000190032003900520029469460007FDF7B9
:108B1000EBFF102000900520694603960195029412
:108B20000007FDF7E1FF11200190029469460095CE
:108B300003941D48FDF7D8FF1E4801906946009632
:108B400002951948FDF7D0FF1B4800900294694632
:108B5000019503941448FDF7C7FFE8026A4651C225
:108B600069461148FDF7C0FF9120000200900520E2
:108B700002946946019503940007FDF7B5FF694625
:108B80000948009702950194FDF7AEFF00220121EC
:108B90000520FEF709FB0520FEF7FAFA07B0F0BD45
:108BA00000100240010600000004005008300000E0
:108BB00000001110000021100836000010B50F4C05
:108BC0000D482060FF20053060600020A060E0605C
:108BD00020616061E0610121206249026062A1615F
:108BE000A0620720E0622046FFF7F8F820680168DD
:108BF00040221143016010BD00300140901400205C
:108C000000B585B014216846FCF7D1FA0E480D492D
:108C10000160E1214902416000218160C160016180
:108C200081610C22C16142610162302141620121F6
:108C3000090381634900C163FFF74AFA01F0D8FBD9
:108C400005B000BD00380140E81400207047000066
:108C500010B5002819DA1A4A03071B0F083B9B08B6
:108C60009B00D2588307DC0EFF23A3409A438B0757
:108C70001B0E8407E40EA3401A43114B0407240F74
:108C8000083CA408A4001A5118E00E4A03231B0252
:108C9000D21883089B00D2588307DC0EFF23A34021
:108CA0009A438B071B0E8407E40EA3401A43054B1F
:108CB000032424021B198408A4001A5110BD0000CB
:108CC0001CED00E000E100E0BFF34F8F04490348D2
:108CD000C860BFF34F8F00BFFDE700000400FA0536
:108CE00000ED00E0F0B587B00A2002F037F97D20F2
:108CF000C00002F04DF9F94C0025A570607B0C28EE
:108D000001D30B2060730122052051020007FDF7FB
:108D1000EEFF0026F248E670F24D00782871F24925
:108D2000A079097840000843E17C89000843E87194
:108D3000A06AE870401CA06260792946A8744200CD
:108D4000B4310846A138FCF719FA06206872E748E2
:108D500000220078A872A07E287328461338217F4D
:108D60000175617F4175607929464000153002F038
:108D7000DFF9607900214000153002F0EBF90220A4
:108D800002F03CF9EE71E673A67201202073E672E0
:108D9000D748FEF7AFF920840546E6706079FCF706
:108DA0006DFCD44AD44BFCF763FB01F08FFD01232B
:108DB00000229B07FCF7AAFAFCF7A6FC0006C10CF0
:108DC000481980B20121C9036084884201D3401A46
:108DD0006084CA4860632079401C2071C448FEF753
:108DE00089F9C04FE0830C373D4642354037AAE150
:108DF000BF48FEF77FF9E083C14E0BE0BC48FEF7A9
:108E000079F980B2E083618C884203D3BD4A891826
:108E1000884206D300210F2002F020F83042E062A1
:108E2000ECD0E06A411C21D040047DD58122D201E2
:108E300000210F2002F051F97D20C00002F0A8F8B7
:108E4000002002F05AF80021102002F007F8410635
:108E5000A448490E264600225030616402F034F8DE
:108E6000A0485030417A0729C1D101E0FFF72CFF1B
:108E70000222A549401DFCF7A5F90028B7D102F050
:108E8000BAF971653446306502F0A2F9F165B06552
:108E9000F0789449401CF0704D310A7968460270B0
:108EA0004979417000880090B18B884274D1974E07
:108EB000288A3080B88A20838D48FEF71BF9E0832A
:108EC00001F0EAFEFF23A16D5B04E06D0022C918EA
:108ED000504100060F0A074379084900080E0902AD
:108EE000216660667F48636D0A30226D02F058F992
:108EF0006079E36D81007B48A26D0818163002F09E
:108F00004FF97848636E1230226E02F049F97548C5
:108F10000821417260790022800072491C3002F001
:108F200007F96079800000E000E100211C3002F0C8
:108F300011F9384602F00BF8012002F05FF82072B8
:108F400002217348FDF7C6FE002826D0002166489E
:108F5000624A0170A8891086E9895186226B626392
:108F6000604A5032D57C2B071B0F032B00D0637453
:108F70002A090027A27401252771584BA5729886EB
:108F8000D986002A18D0574802225F495530FCF78D
:108F900019F9002803D00FE075E00121D7E7514807
:108FA000E573C571606C4F491638C2B26631084628
:108FB0002274D230FCF7E2F8E572208B5549FF307D
:108FC000C33080B2208388420BD9494240182083A5
:108FD00030887D21401C80B2C9003080884200D397
:108FE000378036887D20C000218B70434018A063F5
:108FF00006904948302107784848A77300884843BD
:10900000FCF721FB009030460A214843FCF71BFB8C
:109010000099FCF73DF97F21C905FCF7E0F8FCF762
:109020003BFB80B23C497F1E0880B84200D1E5720C
:10903000A6841420205EFCF70DFB07460391E08B0D
:10904000FCF71CFB364A374BFCF712FA05460E4676
:109050000698FCF7FFFA2A463346FCF7FBF93A4636
:10906000039BFCF753F9FCF72BFBE063608B00F0EC
:1090700075FC207A00286FD100210F2001F0EEFE50
:109080000006F9D568E0FCF7D9FE274A0321115400
:109090001249AA8986000A862348EA894A866038E6
:1090A0003018398B01802049206B303988510D48A8
:1090B000E36D30181630A26D02F072F81A48216B79
:1090C0006038805988423EDD00283CD02046002987
:1090D00039D0009981830221217034E048000020BA
:1090E000C4000020B4110020FC000020D4000020A7
:1090F00060140020B81E85EB51B8CE3FA086010059
:1091000000D02724983A0000E4000020F800002056
:1091100000040050E7030000DA000020DE00002019
:10912000F853E3A59B843E40E01200203246002124
:109130000F2001F0D2FF6079E178401C814202D01B
:10914000002001F0DAFEE08B618C884200D24FE60D
:10915000164A89188842FAD801F09EFD144A002167
:109160000F2001F0BAFFE07B002805D011490B78F1
:1091700048788A78022B0ED00D4A002180320F20C9
:1091800001F0ABFF01210520002249020007FDF795
:10919000AEFD07B0F0BD084BC91C1818FBF7EEFF79
:1091A00002F064F9642001F0F5FB5FE6983A0000F4
:1091B00000D02724EC120020400D00207047000052
:1091C000F0B58DB0B54801900020C0430A9000264C
:1091D0000A2001F0C3FE7D20C00001F0D9FE00206E
:1091E000AF4C0546A070AF4FAF480B90AE48002281
:1091F000C23885730146142001F09AFF0021142023
:1092000001F0A8FF022001F0F9FE00210F2001F07B
:1092100025FE3842E062F8D0E06A0146401C18D0D2
:1092200048047DD58122D20100210F2001F055FF95
:109230000021102001F012FE41069B48490E002239
:10924000801C01F041FE9848801C417A022902D01E
:1092500004E1FFF739FD944802229449C01DFBF751
:10926000B1FF0028F4D101F0C6FF6165206501F06F
:10927000AFFFE165A065002E22D10B988C49008AD2
:10928000088089480126801E808A20838948FDF74E
:1092900031FFE083208B8849FF30C33080B22083C8
:1092A00088420DD949424018814920830888824A62
:1092B000401C80B20B320880904201D3002008800D
:1092C0000B98694682890A80C089488076490422C1
:1092D000C91C0846A238FBF751FFFF22A16D5204BA
:1092E000E06D0023891858410006090A0143084629
:1092F000029101F02CFE029948084000010E000284
:10930000616620666848636D9638226D01F048FFFB
:109310006548E36D9238A26D01F042FF624800E0BB
:109320009EE08E38636E226E01F03AFF5E490022A5
:10933000A0393C2001F0FCFE00213C2001F00AFF96
:10934000012001F05BFE2072A0780121401CA0707A
:109350000520C9030007FCF785FD55487D220088DC
:10936000D200014602905043228B0A398018A06334
:109370000C9052480078A073049008B2E084002852
:1093800003DA7D21C9004018E0844D48302100886F
:109390004843FCF758F905902620205EFCF748F971
:1093A0000599FBF775FF7F21C905FBF718FFFCF74F
:1093B00073F9424980B208800499491E884201D15C
:1093C0000120E0720298A0841420205EFCF742F98C
:1093D00005910690E08BFCF751F93A4A3A4BFCF7BD
:1093E00047F8079104900C98FCF734F9079B049A0E
:1093F000FCF730F8059B069AFBF788FFFCF760F94D
:10940000E063608B00F0AAFA0099019881420DDABE
:1094100000290BD024490422C91C0AA8FBF7AEFE80
:10942000022020700520607200980190207A0028A8
:1094300005D100210F2001F011FD0006F9D5802291
:1094400000210F2001F049FE00206D1CEDB260707C
:10945000032D00D2CAE6002E08D01AE00120F4E75E
:109460001A4A00210F2001F038FEF7E7608B401EFA
:109470000104090C1648618302D00288914201D987
:10948000008860831349608B0988401E4843124955
:1094900008800A98A0830DB0F0BD00003F420F0085
:1094A0004800002000D0272402120020E400002001
:1094B000F800002060140020E7030000DA0000201C
:1094C000DE000020F853E3A59B843E400090272453
:1094D000D0000020CE000020CC000020F8B531499B
:1094E0002F48086001F062FF304C2F486080E08810
:1094F000002801D16420E080208F0A2801D90220B1
:109500002087E08E3C2801D93C20E086284980B2A3
:109510000870284DE08F6871A08FA871A07AE8705C
:10952000A68805212E626981E7883846FBF7E0FDB1
:10953000A88101463046FBF7DBFD8800081886B29B
:109540007D20C0002E817043FCF798F81A4A1B4B0F
:10955000FBF7F6FFFCF7D8F8E8817D206E823946EC
:10956000C000FBF7C5FD28820146C820FBF7C0FDFF
:1095700068830120E882FCF779FCA882EA89104917
:109580001048FDF7BBFD10A0296A00F0D5FFE18867
:1095900011A000F0D1FF218914A000F0CDFFF8BD8B
:1095A00029A400084400002009020000400D00200A
:1095B00000000020C4000020F853E3A59B843E4037
:1095C000FF7F000060140020B1EAC7A949443A2097
:1095D0002564202E0D0A0000CDA8D1B6BCE4B8F455
:1095E0003A202564206D732E0D0A0000B5A5B4CE77
:1095F000CDA8D1B6BBF9D5BECAFDC1BF3A202564FE
:10960000B8F62E0D0A000000F0B5904D85B001208F
:1096100028808F4FC8208F4C3880E079401CE07143
:10962000C00706D0608B411E6183022801D2C8208A
:109630006083608B00F092F90A2001F08FFC7D209E
:10964000C00001F0A5FC02218348FDF743FB002880
:1096500038D00020814980000978824E49000843B3
:109660007F4909780843B072102070727E48C18823
:109670007D20C000FBF73CFD70737C487A49007880
:10968000B07330460B308A780270C9784170411C43
:1096900075482030027ECA70407E087172482230C0
:1096A000027E4A71407E887100220C39152001F03B
:1096B0003FFD0021152001F04DFD022001F09EFC30
:1096C0006B4E03E00120C5E7FEF7A6FF00210F2047
:1096D00001F0C4FB3042E062F6D0E06A411C7DD06C
:1096E00040047CD58122D20100210F2001F0F5FC3D
:1096F0000021102001F0B2FB41065A48490E002219
:109700005030616401F0E0FB564E5036707A1128FB
:1097100065D102225749701DFBF754FD00285ED128
:10972000F01E027969460A7040794870B17A298042
:10973000C820FBF7DDFC3880307B60834E4DB01EC7
:10974000008A2880301F808A20834C48FDF7D2FC95
:1097500080B2E0830390208B4949FF30C33080B250
:10976000208388420CD949424018208328884449E4
:10977000401C80B20B312880884201D30020288011
:109780002D887D20C000218B68434018A063029083
:109790003C48067828460A3800B2A673E0840028C0
:1097A00003DA7D21C9004018E0843888302148431D
:1097B000FBF749FF07462620205EFBF739FF3946B5
:1097C000FBF766FD7F21C905FBF709FDFBF764FF89
:1097D00081B22C48761E0180B14201E033E030E0D6
:1097E00001D10120E072A5841420205EFBF732FF36
:1097F000074601910398FBF741FF234A234BFBF7F0
:1098000037FE05460E460298FBF724FF2A463346EC
:10981000FBF720FE3A46019BFBF778FDFBF750FF74
:10982000E06368460088A0830E480E495030807C73
:1098300060714200633108465130FBF79FFC032002
:10984000207005B0F0BDFFF73FFA0000D400002003
:10985000DE0000204800002000040050C900002065
:10986000CA000020B4110020400D0020000000209C
:1098700000D02724E4000020F8000020601400201D
:10988000E7030000DA000020F853E3A59B843E4084
:1098900070B586B014216846FBF789FC01250F4E90
:1098A000ED03002229463046FDF721FA012000246D
:1098B000019002946946009503943046FDF714F92F
:1098C0000320019002946946009503943046FDF709
:1098D0000BF9022001F05EF806B070BD00040050E4
:1098E00070470000F8B5044600206A461080194D04
:1098F00055222A70AA226A700322AA70661DEE7091
:109900002A716971144A49008918AC712246E81D10
:10991000FBF734FC002007E029186A468978128892
:1099200089186A461180401CB042F5DB611DA81CF5
:10993000FCF7A4F801466846018029190078C8712F
:1099400068464078087221460931024800F0EEFA74
:10995000F8BD0000A0130020400D002010B51B4CE6
:10996000E28A208A6178824201D3101AE082E28A78
:10997000608B134643435B182383132A02D1504361
:1099800040182083208B30214843642164304843B1
:109990000F49E0620968401A0E494018A062FBF7BF
:1099A00059FE0D4A0D4BFBF7CBFDFBF789FE0C4929
:1099B0006062884202DD4A4280186062002801DA53
:1099C0004018606207490968486110BDC400002062
:1099D00084000020F0D8FFFFF853E3A59B843E40AD
:1099E000FF7F000060140020034A1168382389B209
:1099F00099430143116070470030014010B5FDF7F5
:109A000083F910BD10B59AB034216846FBF7CFFB3F
:109A100014210DA8FBF7CBFB1C2112A8FBF7C7FBF9
:109A20001B4801680324E402A143C21489180160A1
:109A3000FDF7CCFB17480169A143016106200090A6
:109A4000FF2001300290012003901020049002209A
:109A5000099040040B90000100240C900A94684681
:109A6000FDF7AAFE0F200D9003200E900F94109486
:109A7000012111940DA8FDF709FD8120129003200A
:109A800080041890149412A8FDF7EAFB1AB010BDD8
:109A9000007000404010024015480068FF2101316D
:109AA0000843134908600846C06812490840104935
:109AB000C86008460068104908400D49086008461B
:109AC00080684008400088600846006801218904D9
:109AD0008843074908600846C068FD210904884397
:109AE0000349C86000200861044805498860704740
:109AF000001002400C40FF88F6FFF6FE0050000800
:109B000000ED00E070B501F0BDF9244C244DA064D7
:109B100004E0FCF715F801F0B5F9A064A842F8D10B
:109B2000207801260525F6032D07002806D00128F8
:109B30000CD0022817D003282CD129E0012231466D
:109B40002846FDF7D4F8FFF75FFD06E00122314615
:109B50002846FDF7CCF8FFF733FB002231462846B4
:109B6000FDF7C5F816E0607A0122401E60723146AA
:109B70002846FDF7BCF8FCF795F900223146284647
:109B8000FDF7B5F8607A002804D10120207001E0CB
:109B9000FFF7A8F801F068F870BD00004800002049
:109BA0003001CADE818CC907C90F002908D00168BD
:109BB0004968012252049143826A1143026851604C
:109BC0000222416A1140022907D101684968D20383
:109BD0009143C26A1143026851600422416A1140F4
:109BE000042907D10168496812049143026B1143AB
:109BF000026851600822416A1140082907D10168B2
:109C0000496812039143426B11430268516010226C
:109C1000416A1140102907D10168896812029143F5
:109C2000826B1143026891602022416A1140202911
:109C300007D10168896812029143C26B114302681F
:109C400091604022416A1140402915D1016849685C
:109C500092039143026C1143026851600122120584
:109C6000016C914208D10168496803225205914371
:109C7000426C1143026851608022416A1140802980
:109C800007D10168496812039143826C114302684D
:109C90005160704738B504460020E067FDF72EF8A4
:109CA0000546206800680821084008280BD11448A0
:109CB0002B46002289040090204600F057FB002824
:109CC00001D0032038BD2068006804210840042822
:109CD0000BD10B482B46002209050090204600F0CE
:109CE00045FB002801D00320ECE720206067A06737
:109CF00000BF00217020015500BF0020E2E70000F6
:109D0000FFFFFF01F8B5184CC826E078002829D1DC
:109D10006079002826D101206071144D686B0027FE
:109D200000281ED0686BC821081A15E01048E168A9
:109D3000405C616988470F480A21008848430E4902
:109D40000880E068401CE060E068C82800DBE7604D
:109D5000696BC820401A761EE168814201D0002E4E
:109D6000E4DC6771F8BD0000300000200000024014
:109D7000780C0020D4000020E000002070B5224CB8
:109D8000E07800283FD1207900283CD101202071C3
:109D90001E4EF16900250906002933DA2156625763
:109DA00091420AD1F06940062CD5A079002829D02B
:109DB000A5712089401C208124E0A179002903D1CC
:109DC000A0710A2000F0EDFD00202056CC21484370
:109DD0000F494218206912181279B262401C002201
:109DE0002061A256CC235A43895881420ADC25615E
:109DF0002078401C207020780E2800D12570A07893
:109E0000401CA070257170BD30000020003801405A
:109E10005001002070B50546AC6A00215A2001535C
:109E2000522001532046FEF76CF870BDF8B5054688
:109E3000AC6A666FA76F2068806880210840802820
:109E400007D1212E05D1002152200153204600F0D8
:109E500064F82068806840210840402807D1222FFC
:109E600005D100215A200153204600F034F8E06F5C
:109E700010210843E0672046FEF743F8F8BD70B5AF
:109E80000546AC6A2868006820210840002817D1E0
:109E900000215A20015320680068FF2101318843C6
:109EA0002168086020688068400840002168886058
:109EB0002068806840218843216888602020A0674E
:109EC0002046FEF723FA70BD70B50446A56A284601
:109ED000FEF71DFA70BD01680968FF222132914327
:109EE0000268116001688968490849000268916048
:109EF0002021816700210166704710B50446206863
:109F000000684021884321680860202060670020A5
:109F100060662046FEF77CFA10BD01680968C02221
:109F200091430268116020214167704770B5164C5B
:109F3000E278002A0CD12279002A09D10122E270AC
:109F40000025C82903DC0222A256002A01DCE570A4
:109F500070BD0123E356CC2253430C4AD150012358
:109F6000E356CC2673439B180A460146181DFBF79F
:109F700005F96078401C607060780E2800D165702B
:109F8000A078401EA070E2E73000002050010020C1
:109F9000F0B587B0044610200490002500200390FF
:109FA0000026E7492068884200D100E000BF21690F
:109FB000A068084361690843E169084307462068CF
:109FC0000068E0490840384321680860206840681C
:109FD000032109038843E168084321684860A769B1
:109FE000D7492068884201D0206A074320688068EA
:109FF0000B210902884338432168886000BFD24999
:10A00000206888421CD1D148C0688007800F002892
:10A0100006D001280AD0022805D003280CD108E078
:10A02000012004900BE00220049008E0042004903A
:10A0300005E00820049002E01020049000BF46E0F4
:10A04000C349206888421CD1C048C0680C21084020
:10A05000002806D004280AD0082805D00C280CD1E6
:10A0600008E0002004900BE00220049008E00420A7
:10A07000049005E00820049002E01020049000BF46
:10A0800025E0AF49206888421FD1B048C06803214D
:10A0900089020840002808D001218902401A0AD00C
:10A0A000401A05D0401A0CD108E0002004900BE0C3
:10A0B0000220049008E00420049005E008200490A9
:10A0C00002E01020049000BF01E01020049000BFC7
:10A0D0009B492068884256D1049804281AD004DC91
:10A0E000002807D002281CD108E0082816D0102824
:10A0F00017D117E0FDF7D4FA064616E0934840382A
:10A100000068102108400009002801D0914E00E0AD
:10A11000914E0AE0FDF7E8FA064606E00126F6034E
:10A1200003E000BF0120039000BF00BF002E0AD053
:10A13000606841004018B04203D860680003B04234
:10A1400002D201200390F4E0606802903046FF21C3
:10A15000013100F018FA6268520800238018594152
:10A1600001910090029AFAF7D9FF054603200002F8
:10A17000854205D37948854202D82068C560D8E079
:10A1800001200390D5E00121C903E06988426FD125
:10A19000049804283CD006DC002809D0012813D0FC
:10A1A00002284AD11CE008283ED0102845D145E0BD
:10A1B000FDF776FA4000616849084018029061682E
:10A1C000FAF796FF85B23CE0FDF77CFA4000616843
:10A1D0004908401802906168FAF78AFF85B230E0BA
:10A1E0005A4840380068102108400009002807D06C
:10A1F00061684A085A4BD018FAF77AFF85B206E030
:10A2000061684A08574BD018FAF772FF85B218E018
:10A21000FDF76AFA400061684908401802906168D9
:10A22000FAF766FF85B20CE061684A0801231B0457
:10A23000D018FAF75DFF85B203E000BF012003905C
:10A2400000BF00BF102D0FD3474885420CD84648A9
:10A250000F38284005902807400F059908430590BE
:10A2600005982168C86064E00120039061E0FFE781
:10A27000049804283AD006DC002809D0012812D01E
:10A28000022847D11AE008283BD0102842D142E0EA
:10A29000FDF706FA61684908401802906168FAF70C
:10A2A00027FF85B23AE0FDF70DFA616849084018CA
:10A2B00002906168FAF71CFF85B22FE0234840380E
:10A2C0000068102108400009002807D061684A088A
:10A2D000204BD018FAF70CFF85B206E061684A08F7
:10A2E0001D4BD018FAF704FF85B217E0FDF7FCF913
:10A2F00061684908401802906168FAF7F9FE85B272
:10A300000CE061684A080123DB03D018FAF7F0FE7D
:10A3100085B203E000BF0120039000BF00BF102DF5
:10A3200005D31148854202D82068C56001E00120AC
:10A330000390002020666066039807B0F0BD00001F
:10A3400000480040F369FFEF003801404010024030
:10A350000044004000093D000024F400FFFF0F000E
:10A3600000127A000048E801FFFF0000FFB581B04D
:10A3700004460D4617460A9E22E0701C00281FD096
:10A38000FCF7BCFC0499401AB04201D8002E17D14A
:10A3900020680068FF21A131884321680860206897
:10A3A0008068400840002168886020206067A067BE
:10A3B00000BF00217020015500BF032005B0F0BD93
:10A3C0002068C0692840A84201D1012000E0002097
:10A3D000B842D2D00020F1E710B504491020096836
:10A3E00008620248FDF78EFD10BD0000E814002051
:10A3F00001490D20887070473000002010B50748D3
:10A400000A22018A51438183FEF716FBFEF7F8FB0F
:10A41000C82203490348FDF705FF10BDC400002012
:10A42000780C0020E8140020F8B53E4C0023217879
:10A430003D4A1D46082910D0072947D0062950D08B
:10A44000052952D0042953D0032954D0002956D0CD
:10A45000012958D002295AD05BE0A17800264A1F72
:10A4600004E0314FBF5DFB189BB2761C9642F8DBCF
:10A47000667927799A195118E3786278C91889188A
:10A48000C9194018C0430006000E1AD1012E14D07D
:10A49000022E16D125482449C018FAF76FFE00F0A5
:10A4A000E5FF642000F076FABFF34F8F2149204882
:10A4B000C860BFF34F8F00BFFDE759081046FFF794
:10A4C00011FA2570E570A570A571F8BDA1795054F9
:10A4D000491CC8B2A071A178491F8842F5D1082053
:10A4E00001E0607007202070F8BDE0700620FAE7F8
:10A4F00060710520F7E7A070E5700420F3E75528A8
:10A5000007D10120EFE7AA2803D10220EBE70328B7
:10A5100003D02570E570A570F8BD03202070207170
:10A52000F8BD0000BB0000203C130020400D0020BF
:10A530000400FA0500ED00E00FB410B503A9044BC8
:10A54000044A029800F01AF910BC08BC04B018477D
:10A55000B9B10008100100202021020C01D0102107
:10A560001046020A01D010460839020901D01046EF
:10A57000091F820801D01046891E420801D0881E9A
:10A580007047081A7047F8B582B28BB2040C0D0CF4
:10A5900010465843002126465E43370C3604801986
:10A5A000794116466E43370C3604801979412646A8
:10A5B0006E438919F8BD30B47446641E2578641C56
:10A5C000AB4200D21D46635D5B00E31830BC184708
:10A5D00002E008C8121F08C1002AFAD1704770476C
:10A5E000002001E001C1121F002AFBD1704708B50D
:10A5F0000021684601706B46012202212C2000F0E8
:10A600007BFD0221684601706B4601222C2000F080
:10A6100073FD08BD38B504466D20694608706B4669
:10A62000012207492E2000F067FD0649002C01D0C9
:10A63000054A00E0054A2E2000F044FD38BD000028
:10A6400006080000061800000706000007160000B4
:10A6500038B504466B4602220021362000F018FC73
:10A66000B3212300FFF7A7FF0E0F08153A3A3A3A35
:10A670001C273A3A2F34483A002168460170407846
:10A680004108490014E06946087880088000401CB1
:10A6900004E06946087880088000801C08701DE08E
:10A6A000684602780A4048320270417880200143AF
:10A6B0006846417012E0684602780A4002704078AD
:10A6C0004106490EF4E7694648780221084303E051
:10A6D00069464878FD210840694648706B4601226A
:10A6E0000021362000F008FD012200AB1146362083
:10A6F000013300F001FD38BD69460878CF210840DC
:10A7000069462030CAE708B5032168464170012137
:10A7100001706B4602220021362000F0EDFC012280
:10A72000D20306212D2000F0CDFC012000F032F9EB
:10A730000120FFF78DFF08BD08B5020A69464A707F
:10A7400008706B46022204212D2000F0D5FC032066
:10A75000694608706B46012206212D2000F0CCFCD2
:10A760000020694608706B46012206212D2000F06A
:10A77000C3FC0A212D2000F071FB08BDFFB58DB090
:10A780000446002506E025280AD0109A0F99904724
:10A79000641C6D1C20780028F5D1284611B0F0BD4E
:10A7A00000270121484A009700E00743641C2378F2
:10A7B0000846203B98401042F7D120782E2817D128
:10A7C000042007436078641C2A280CD10E98641C6E
:10A7D00002C800910E900BE000990A2251433039D3
:10A7E0004018641C00902078014630390929F3D9BB
:10A7F00020780028D1D0642808D0692806D0752890
:10A800001ED0109A0F9990476D1C5BE00A200E999C
:10A81000019001C90E91002802DA40422D2102E088
:10A82000390504D52B216A461172012103E0F9078D
:10A8300004D02021F7E70BAE0B910DE00021FAE7E1
:10A840000A200E99019001C90E91F7E70199FAF7D4
:10A850004FFC3031761E31700028F7D103A8801BE1
:10A8600020300190780701D5009801E00120009088
:10A870000199884201DD401A00E000200027009085
:10A8800006E002A8109AC05D0F9990476D1C7F1CCE
:10A890000B988742F5DB04E0109A30200F9990471F
:10A8A0006D1C0099481E00900029F5DC05E0307809
:10A8B000109A761C0F9990476D1C0199481E0190C3
:10A8C0000029F4DC641C65E709280100F8B54A009A
:10A8D0002B4B520DD6182B4A0C460546142E2BDA5C
:10A8E000002E12DA284BFAF711FD00221346FBF76F
:10A8F00037F840D2002C03DA0124E40700253AE0BF
:10A900002046284337D0214C14E0214F0B46F74016
:10A910003B402B4331D01C4BFAF7F8FC0022134686
:10A92000FBF71EF827D2002C03DD01200005F040C4
:10A930000419BC4300251EE0332E1EDC33460027DD
:10A94000143BFF43DF40384217D00F4BFAF788FD26
:10A9500000221346FBF704F80DD2002C0ADD142E5A
:10A960000CD03420811B012088404019A84200D21D
:10A97000641C0546BD4321462846F8BD641CF9E722
:10A9800001FCFFFF9C7500883CE4377E0000F03F2F
:10A99000FFFF0F007D2110B5C900484300F001F80A
:10A9A00010BD002140E000BF00BF00BF00BF00BFDE
:10A9B00000BF00BF00BF00BF00BF00BF00BF00BF9F
:10A9C00000BF00BF00BF00BF00BF00BF00BF00BF8F
:10A9D00000BF00BF00BF00BF00BF00BF00BF00BF7F
:10A9E00000BF00BF00BF00BF00BF00BF00BF00BF6F
:10A9F00000BF00BF00BF00BF00BF00BF00BF00BF5F
:10AA000000BF00BF00BF00BF00BF00BF00BF00BF4E
:10AA100000BF00BF00BF00BF00BF00BF00BF00BF3E
:10AA200000BF00BF00BF491C8142BCD3704700007B
:10AA3000FEB5044600200190009060797349400003
:10AA40000E5A61782578491E7148CFB20163042DF2
:10AA500077D0072D75D000210291217801736C49C0
:10AA6000E379012292058969002B6CD091438161C1
:10AA70006748217A4173217A82698907890B0A43E1
:10AA800082610021042000F028FB324661492E201B
:10AA900000F018FB3846FFF7BDFD5F4E0522705DE4
:10AAA000810040185D49431807212B2000F024FB4A
:10AAB0005B49029801220B180B21282000F01CFB97
:10AAC000705D584980000A580C21282000F005FBD1
:10AAD000E079554980004018A1794900425A022185
:10AAE000272000F0EFFA51487E00825B04212720E6
:10AAF00000F0E8FAE079002829D0A07804282CD0CA
:10AB000028206946087220220621272000F0DAFA60
:10AB100002AB01222621272000F0EEFA4449380139
:10AB20004018E178890042580821272000F0D5FA22
:10AB3000A17A601C627A0902114313D016E000E08A
:10AB400001E0012188E71143F608816190E7642262
:10AB50000621272000F0B6FAE0E7102069460872C7
:10AB60000246D1E733490172090A4172417A007AFB
:10AB70000A0202432021272000F0A4FA2E4F0C21C4
:10AB800023203A6800F0A9FAF019828804212320D2
:10AB900000F098FAA07900280BD0E079274901222B
:10ABA00043180021212000F0A7FA03200190012082
:10ABB00000902A07120F10010243607800218007DD
:10ABC000000B024301980005024300984004024331
:10ABD0002079C006400902436079C00602431F2065
:10ABE00000F07BFAA078617801230843020408484A
:10ABF000DB030261E179490319430A430261002141
:10AC0000082000F06AFA0020FEBD000038B50008F8
:10AC10001401002004280000E0B400080100002016
:10AC20001F000020E8B4000808B5000814B50008AB
:10AC300018B500084110000000B5000821000020F0
:10AC400038B50C4607498A8B002102432C2000F0BE
:10AC500039FA684604706B46012206212C2000F068
:10AC60004BFA38BD1401002010B5FFF7C0FC10BD31
:10AC700010B504460421362000F0F0F80121C90285
:10AC8000002C01D0084300E088430246042136200E
:10AC900000F023FA10BD000038B540206946087066
:10ACA00000210E2000F0DAF80446002211460E20A2
:10ACB00000F013FA6B46012200210D2000F01CFA6F
:10ACC000074A00210F2000F008FA00F0E1F92246BF
:10ACD00000210E2000F001FA02480021017338BD66
:10ACE000F8FF2724340100207CB50546042069467E
:10ACF00008704B4C0020607521462031206348715C
:10AD00000873A0836063A06300F0BCF8454E206028
:10AD100002E000F0B7F82060B042FAD10020FFF75F
:10AD200097FC41480078242801D9243806E0062100
:10AD3000FAF7DEF90622101A400108430206010460
:10AD40000A4301020A43024300211E2000F0C5F914
:10AD50006B4601220021242000F0CEF91E20FFF7CF
:10AD6000EBFC86B2300AA0730420FFF7E5FC000676
:10AD7000000E0DD002206946087101AB012212219C
:10AD80002D2000F0B9F9A08B012109030843A0830D
:10AD900000F078F820600620FFF7CEFC6060072006
:10ADA000FFF7CAFCA060F006C00E207501D110208C
:10ADB0002075C0B200F0DCF9E80707D0FFF7A3FC6C
:10ADC000A08B0121C9020843A0830AE00521362097
:10ADD00000F02EF81549084002460521362000F003
:10ADE00071F90120FFF734FC0021042000F036F84F
:10ADF000A0610021262000F031F8152189030843C5
:10AE000002460021262000F068F900222621362083
:10AE100000F058F900F036F8206000207CBD0000FA
:10AE2000140100203001CADE00000020FFFD0000F8
:10AE300038B5094C89B280B26B46022200F028F87E
:10AE4000002806D168464078010268460078081854
:10AE500084B2204638BD0000FFFF000038B5002452
:10AE6000E44389B280B26B46042200F011F8002856
:10AE700006D103216846435C2202D418491EFAD544
:10AE8000204638BD10B500210846FFF7E7FF10BD8A
:10AE900038B5002909D0402420436C462070C8B240
:10AEA0007F2906D8607002200AE0694608700120F8
:10AEB00006E0802420436C466070C809A07003201F
:10AEC000694600F0ADFA38BD10B5144603460A468F
:10AED00021461120FFF7DCFF10BD10B50346052207
:10AEE00000211520FFF7D4FF10BD10B50346052241
:10AEF00000211720FFF7CCFF10BD38B50546002014
:10AF00006946087000F0C4F8FF2401342246002D81
:10AF100001D00322120200210D2000F0D3F8002DF1
:10AF200013D06B46012203210F20FFF7B1FF6846C3
:10AF30000078000709D5FFF7AFFE224600210D205B
:10AF400000F0C0F80020C04338BD002038BD10B567
:10AF5000024601210A2000F0C0F810BD10B50446D9
:10AF600000211A20FFF77AFF000D22030005120BC3
:10AF7000024300211A2000F0B0F810BD10B50246BF
:10AF800002492E2000F09EF810BD000004180000B9
:10AF9000F8B505466B46012203210420FFF778FF30
:10AFA0000126114C3607002D0DD02A4600210C2019
:10AFB00000F088F86946087810210843694608704F
:10AFC000A069304307E069460878EF2108406946E8
:10AFD0000870A069B0430B46A06101220321042040
:10AFE00000F08AF8F8BD00001401002010B50246F8
:10AFF0000021182000F066F810BD0000F8B50746E3
:10B00000002568460570B807204C2E4600280ADA4D
:10B010008020694608706B46012200210D2000F057
:10B020006BF801202073F8076946087821D00621C3
:10B030000843694608706B46012200210D2000F08C
:10B040005BF803210F20FFF7F3FE8121C9000842BE
:10B0500019D04020694608706B46012200210D205E
:10B0600000F04AF80020FFF703FE00252673ED43A9
:10B0700009E002210843694608706B46012200215D
:10B080000D2000F039F82846F8BD000034010020FA
:10B090001CB56B46012203210F20FFF7F9FE68461D
:10B0A00000784022C1091040C9014000814208D007
:10B0B000012069460871024601AB03210D2000F012
:10B0C0001BF81CBD08B56B461A70120A5A7089B27B
:10B0D00080B2022200F010F808BD38B500236C469B
:10B0E000E254120A5B1C042BFADB89B280B22346BD
:10B0F000042200F001F838BD38B58024002909D0B9
:10B10000C02528436D462870C8B27F2907D86870CB
:10B11000022009E0204369460870012004E0204332
:10B120006870C809A8700320694600F0B5F938BDF9
:10B1300010B51446012312189B029A4202D900202E
:10B14000C04310BD0B46821E21460920FFF7D4FFE5
:10B15000002010BD10B5054A8905126901430A4354
:10B1600000210820FFF7B9FF002010BD14010020C6
:10B1700038B504466B4601220E212B20FFF788FECE
:10B1800068460078E10640094001C90E014368465F
:10B1900001706B4601220E212B20FFF7ADFF38BD59
:10B1A00010B5002142541C06120A22431B0A491CF6
:10B1B0000429F7DB10BD000013B501231A466946C8
:10B1C0000248FDF7A5F800981CBD0000E814002017
:10B1D0007CB5002425466846FFF77FFE04206946BB
:10B1E000220E2D02154322020C5C1443401EF7D59B
:10B1F000204629467CBD7CB5002425466846FFF7DD
:10B2000074FE04206946220E2D02154322020C5CB6
:10B210001443401EF7D5204629467CBDFBF77CFD34
:10B22000FEF7F0FBFDF71CFC3B493C48002522C023
:10B2300005608561C5613A490562C1600838FBF760
:10B24000D1FEFDF7F9FBFDF7DBFCFDF7B7FCFDF7E1
:10B25000BFFB052601223607D1033046FBF747FD29
:10B26000FEF73CF9FDF78AFAFAF76AFCFAF738FCC0
:10B270000721B015FFF7E4FC2A4C0A21208A01229D
:10B280004843A083170339463046FBF730FD234877
:10B29000C82225498830FCF7C5FF244E20790028B4
:10B2A00036D0FEF7AFFB2571FAF78EFE20700F281F
:10B2B00009D9012239463046FBF719FDFEF722FC79
:10B2C0000022394609E0012251033046FBF70FFD09
:10B2D000FEF718FC0022012149033046FBF707FD69
:10B2E000FDF79AF9A08B002801D0401EA0831048DA
:10B2F000A18B00780843D1D10121C9023046FBF768
:10B30000E9FC0028CAD101210846FBF785FFC5E703
:10B31000FDF782F9C2E70000007C004060140020C5
:10B32000FFFF0000C4000020780C00200004005043
:10B330003600002010B586B01748FBF7AEFD14218B
:10B340006846F9F734FF154800900320019000206B
:10B350000290052069460007FBF7C6FB69461048C6
:10B36000FBF7C2FB69460F48FBF7BEFB012108460D
:10B37000FBF752FFFF2401342046FBF71FFF0A4969
:10B3800008680422104308602046FBF729FFFBF7FA
:10B390002FFF06B010BD000060140020FFFF00006A
:10B3A00000040050000800500070004010B5012259
:10B3B000920218491848FAF74FFC164817490288B4
:10B3C0008A4225D001807D21C90081804910C18039
:10B3D0000A21018100211E224181D2438281012262
:10B3E000C2810184018241828182C1820183818381
:10B3F0001E23C38602230387782343878287C2875D
:10B4000002464032118451849184C18300F02EF8A9
:10B4100010BD0000400D002000FC0008AA550000EF
:10B42000F0B58C4600251026052109078E620E4CCA
:10B4300008E067467F5DE760A768FF07FCD0E76824
:10B440001F706D1C8542F4DB0020074606E0E760B4
:10B45000A568ED07FCD0E5681D54401C9042F6D36A
:10B460008E610020F0BD00000030014070B572B662
:10B470000124074DA40221462846FAF7D3FB0028F1
:10B4800004D0224603492846FAF7BCFC62B670BDD8
:10B4900000FC0008400D0020F0B50025102605270F
:10B4A0009C463F070B46BE620C4C06E0595DE160CE
:10B4B000A168C907FCD0E1686D1C8542F6DB00205D
:10B4C00007E06146095CE160A168C907FCD0E1685A
:10B4D000401C9042F5D3BE610020F0BD0030014019
:10B4E0000000010203040005405C0000A05C0400B1
:10B4F000C06C0800805C0400E03F1E00E07D1E0080
:10B5000007A9022570889B880A0016000100060022
:10B510000100020087008D002D001A3152001A33FD
:10B520009A001A351D011A376B003B31BE003B33C0
:10B530005E013B3596023B37000099599959EB5112
:10B540008F421E45142E0080EB51F5283333E13A2B
:10B55000703DE13AC235852BC2353333C235C23531
:10B56000AE47E13A5138A3305138000000000000E6
:10B5700000000102030406070809000000000102A0
:10B580000304030406080C1018203000ACB50008B2
:10B590000000002014010000D0A50008C0B600087B
:10B5A00014010020FC180000E0A5000800070400BA
:10B5B000091E0805400826091040085608054008DD
:10B5C000261D040008BE1D040008BED8BC4010089B
:10B5D000010000000000C842000000000000000060
:10B5E000000000000000000000000000000000005B
:10B5F000000000000100000000000000000000004A
:10B6000000000000000000005C12000000000000CC
:10B61000000000000000000000000000000000002A
:10B62000000000000000000000000000000000001A
:10B63000000000000000000000000000000000000A
:10B6400000000000000000000000000000000000FA
:10B6500000000000000000000000000002020400E2
:10B660000909010200810000000000000100000043
:10B6700000080000000000000000000000000000C2
:10B6800000000000000000000000000000000000BA
:10B6900000000000000000000000000000000000AA
:10B6A000000000000000000000000000000000009A
:10B6B000000000000000000000002000000000006A
:04000005080050C1DE
:00000001FF
